:100000000C9446000C9463000C9463000C94630001
:100010000C9463000C9463000C9463000C946300D4
:100020000C9463000C9463000C9463000C946300C4
:100030000C9463000C9463000C9463000C946300B4
:100040000C9463000C9463000C9463000C946300A4
:100050000C9463000C9463000C9463000C94630094
:100060000C9463000C9463000C9463000C94630084
:100070000C9463000C9463000C9463000C94630074
:100080000C9463000C9463000C94630011241FBE55
:10009000CFEFD0E1DEBFCDBF11E0A0E0B1E0E8EBF3
:1000A000F6E300E00BBF02C007900D92AC38B10739
:1000B000D9F711E0ACE8B1E001C01D92AE38B1074C
:1000C000E1F70C9465000C9400000F931F93CF93FD
:1000D000DF93CDB7DEB7CA50D1400FB6F894DEBF7C
:1000E0000FBECDBFEAE3F0E08FEF8083E7E3F0E0FF
:1000F0008FEF8083E1E6F0E01082E8E3F0E0108229
:10010000E2E6F0E01082CE018D519F4FCC5FDE4FD2
:1001100099838883C450D140CC5FDE4FA881B981D8
:10012000C450D140CA5FDE4FB983A883C650D140C6
:10013000EFE6F1E0C85FDE4FF983E883C850D140B5
:10014000FDE0C65FDE4FF883CA50D140C85FDE4F86
:10015000A881B981C850D1400C90C85FDE4FE881BA
:10016000F981C850D1403196C85FDE4FF983E883EA
:10017000C850D140CA5FDE4FA881B981C650D14076
:100180000C92CA5FDE4FE881F981C650D1403196AA
:10019000CA5FDE4FF983E883C650D140C65FDE4FA9
:1001A000F881CA50D140F150C65FDE4FF883CA5083
:1001B000D140C65FDE4F8881CA50D140882331F6D6
:1001C00088E0CC5FDE4FE881F981C450D1403D9694
:1001D000DF01982F1D929A95E9F70E94A209FE016E
:1001E000E153FF4F80E090E0A0EAB0E48083918388
:1001F000A283B3838E010B521F4FFE01E153FF4FC9
:1002000026E636E646E655E4608171818281938177
:100210000E945C13DC01CB01F80180839183A283EF
:10022000B383FE01EB52FF4F20E030E040E85FE394
:1002300060817181828193810E94E61488230CF091
:1002400008C0FE01ED52FF4F81E090E09183808372
:1002500027C0FE01EB52FF4F20E03FEF4FE757E48E
:1002600060817181828193810E947A1418160CF04A
:1002700006C0FE01ED52FF4F1182108211C08E01A7
:100280000D521F4FFE01EB52FF4F60817181828141
:1002900093810E94AB11DC01CB01F8019183808333
:1002A000DE01A353BF4FFE01ED52FF4F80819181CC
:1002B0008D939C93FE01E353FF4F808191810197C1
:1002C000F1F7FE01E353FF4F918380830E94BF0E3D
:1002D0000E94B109FE01E752FF4F1182108283C0D4
:1002E000FE01ED53FF4F80E090E0A0E2B1E4808397
:1002F0009183A283B3838E0107531F4FFE01ED53F9
:10030000FF4F26E636E646E655E46081718182813C
:1003100093810E945C13DC01CB01F80180839183FF
:10032000A283B383FE01E753FF4F20E030E040E8B3
:100330005FE360817181828193810E94E61488234A
:100340000CF008C0FE01E953FF4F81E090E091837B
:10035000808327C0FE01E753FF4F20E03FEF4FE7C8
:1003600057E460817181828193810E947A1418160A
:100370000CF006C0FE01E953FF4F1182108211C03C
:100380008E0109531F4FFE01E753FF4F60817181BA
:10039000828193810E94AB11DC01CB01F801918332
:1003A0008083DE01AF53BF4FFE01E953FF4F8081D1
:1003B00091818D939C93FE01EF53FF4F808191813A
:1003C0000197F1F7FE01EF53FF4F91838083DE0128
:1003D000A752BF4FFE01E752FF4F808191810196E6
:1003E00011969C938E93FE01E752FF4F808191817D
:1003F0008A3091050CF474CFE7E2F0E083E6808365
:10040000FE01E954FF4F80E090E0A0EAB0E4808371
:100410009183A283B3838E0103541F4FFE01E954DD
:10042000FF4F26E636E646E655E46081718182811B
:1004300093810E945C13DC01CB01F80180839183DE
:10044000A283B383FE01E354FF4F20E030E040E895
:100450005FE360817181828193810E94E614882329
:100460000CF008C0FE01E554FF4F81E090E091835D
:10047000808327C0FE01E354FF4F20E03FEF4FE7AA
:1004800057E460817181828193810E947A141816E9
:100490000CF006C0FE01E554FF4F1182108211C01E
:1004A0008E0105541F4FFE01E354FF4F608171819F
:1004B000828193810E94AB11DC01CB01F801918311
:1004C0008083DE01AB54BF4FFE01E554FF4F8081B6
:1004D00091818D939C93FE01EB54FF4F808191811C
:1004E0000197F1F7FE01EB54FF4F91838083E5E222
:1004F000F0E08081FE01E552FF4F992791838083D0
:10050000DE01A552BF4FFE01E552FF4F8081918170
:100510008C599F4F8D939C93DE01AF51BF4FFE01CD
:10052000E552FF4F808191818D939C93FE01EF51A5
:10053000FF4F808191819F938F938CE691E09F93F1
:100540008F93CE018D519F4F9F938F930E9496174B
:100550008DB79EB706960FB6F8949EBF0FBE8DBF9F
:10056000FE01E555FF4F80E090E0A0EAB0E4808313
:100570009183A283B3838E010F541F4FFE01E55573
:10058000FF4F26E636E646E655E4608171818281BA
:1005900093810E945C13DC01CB01F801808391837D
:1005A000A283B383FE01EF54FF4F20E030E040E828
:1005B0005FE360817181828193810E94E6148823C8
:1005C0000CF008C0FE01E155FF4F81E090E09183FF
:1005D000808327C0FE01EF54FF4F20E03FEF4FE73D
:1005E00057E460817181828193810E947A14181688
:1005F0000CF006C0FE01E155FF4F1182108211C0C0
:100600008E0101551F4FFE01EF54FF4F6081718134
:10061000828193810E94AB11DC01CB01F8019183AF
:100620008083DE01A755BF4FFE01E155FF4F80815A
:1006300091818D939C93FE01E755FF4F80819181BD
:100640000197F1F7FE01E755FF4F9183808365E045
:1006500070E082E090E00E94A50FFE01E156FF4F9E
:1006600080E090E0A0EAB0E480839183A283B3832A
:100670008E010B551F4FFE01E156FF4F26E636E671
:1006800046E655E460817181828193810E945C130A
:10069000DC01CB01F80180839183A283B383FE0147
:1006A000EB55FF4F20E030E040E85FE3608171816F
:1006B000828193810E94E61488230CF008C0FE0119
:1006C000ED55FF4F81E090E09183808327C0FE01CC
:1006D000EB55FF4F20E03FEF4FE757E4608171811A
:1006E000828193810E947A1418160CF006C0FE01D4
:1006F000ED55FF4F1182108211C08E010D551F4F15
:10070000FE01EB55FF4F60817181828193810E94D0
:10071000AB11DC01CB01F80191838083DE01A3568C
:10072000BF4FFE01ED55FF4F808191818D939C93CA
:10073000FE01E356FF4F808191810197F1F7FE01A1
:10074000E356FF4F91838083CE018D519F4F0E94CE
:10075000800FFE01ED56FF4F80E090E0A0EAB0E48C
:1007600080839183A283B3838E0107561F4FFE01BE
:10077000ED56FF4F26E636E646E655E46081718188
:10078000828193810E945C13DC01CB01F80180839C
:100790009183A283B383FE01E756FF4F20E030E050
:1007A00040E85FE360817181828193810E94E61459
:1007B00088230CF008C0FE01E956FF4F81E090E06D
:1007C0009183808327C0FE01E756FF4F20E03FEF73
:1007D0004FE757E460817181828193810E947A148E
:1007E00018160CF006C0FE01E956FF4F1182108268
:1007F00011C08E0109561F4FFE01E756FF4F608161
:100800007181828193810E94AB11DC01CB01F801DF
:1008100091838083DE01AF56BF4FFE01E956FF4F43
:10082000808191818D939C93FE01EF56FF4F8081D3
:1008300091810197F1F7FE01EF56FF4F918380837D
:10084000E7E2F0E082E68083FE01E957FF4F80E0B7
:1008500090E0A0EAB0E480839183A283B3838E0109
:1008600003571F4FFE01E957FF4F26E636E646E6DF
:1008700055E460817181828193810E945C13DC0167
:10088000CB01F80180839183A283B383FE01E357F8
:10089000FF4F20E030E040E85FE3608171818281BA
:1008A00093810E94E61488230CF008C0FE01E557EE
:1008B000FF4F81E090E09183808327C0FE01E357E2
:1008C000FF4F20E03FEF4FE757E460817181828165
:1008D00093810E947A1418160CF006C0FE01E557A9
:1008E000FF4F1182108211C08E0105571F4FFE016C
:1008F000E357FF4F60817181828193810E94AB1128
:10090000DC01CB01F80191838083DE01AB57BF4F3F
:10091000FE01E557FF4F808191818D939C93FE01ED
:10092000EB57FF4F808191810197F1F7FE01EB5763
:10093000FF4F91838083E5E2F0E08081FE01E55284
:10094000FF4F992791838083DE01A552BF4FFE019F
:10095000E552FF4F808191818C599F4F8D939C93DD
:10096000DE01AF51BF4FFE01E552FF4F8081918103
:100970008D939C93FE01EF51FF4F808191819F9356
:100980008F938CE691E09F938F93CE0188509F4F79
:100990009F938F930E9496178DB79EB706960FB6BA
:1009A000F8949EBF0FBE8DBFFE01E558FF4F80E05B
:1009B00090E0A0EAB0E480839183A283B3838E01A8
:1009C0000F571F4FFE01E558FF4F26E636E646E675
:1009D00055E460817181828193810E945C13DC0106
:1009E000CB01F80180839183A283B383FE01EF578B
:1009F000FF4F20E030E040E85FE360817181828159
:100A000093810E94E61488230CF008C0FE01E1588F
:100A1000FF4F81E090E09183808327C0FE01EF5774
:100A2000FF4F20E03FEF4FE757E460817181828103
:100A300093810E947A1418160CF006C0FE01E1584A
:100A4000FF4F1182108211C08E0101581F4FFE010D
:100A5000EF57FF4F60817181828193810E94AB11BA
:100A6000DC01CB01F80191838083DE01A758BF4FE1
:100A7000FE01E158FF4F808191818D939C93FE018F
:100A8000E758FF4F808191810197F1F7FE01E75808
:100A9000FF4F918380836FE070E082E090E00E94DE
:100AA000A50FFE01E159FF4F80E090E0A0EAB0E41D
:100AB00080839183A283B3838E010B581F4FFE0165
:100AC000E159FF4F26E636E646E655E4608171813E
:100AD000828193810E945C13DC01CB01F801808349
:100AE0009183A283B383FE01EB58FF4F20E030E0F7
:100AF00040E85FE360817181828193810E94E61406
:100B000088230CF008C0FE01ED58FF4F81E090E013
:100B10009183808327C0FE01EB58FF4F20E03FEF19
:100B20004FE757E460817181828193810E947A143A
:100B300018160CF006C0FE01ED58FF4F118210820E
:100B400011C08E010D581F4FFE01EB58FF4F608101
:100B50007181828193810E94AB11DC01CB01F8018C
:100B600091838083DE01A359BF4FFE01ED58FF4FF3
:100B7000808191818D939C93FE01E359FF4F808189
:100B800091810197F1F7FE01E359FF4F9183808333
:100B9000CE0188509F4F0E94800FFE01ED59FF4FFC
:100BA00080E090E0A0EAB0E480839183A283B383E5
:100BB0008E0107591F4FFE01ED59FF4F26E636E61D
:100BC00046E655E460817181828193810E945C13C5
:100BD000DC01CB01F80180839183A283B383FE0102
:100BE000E759FF4F20E030E040E85FE3608171812A
:100BF000828193810E94E61488230CF008C0FE01D4
:100C0000E959FF4F81E090E09183808327C0FE0186
:100C1000E759FF4F20E03FEF4FE757E460817181D4
:100C2000828193810E947A1418160CF006C0FE018E
:100C3000E959FF4F1182108211C08E0109591F4FCF
:100C4000FE01E759FF4F60817181828193810E948B
:100C5000AB11DC01CB01F80191838083DE01AF5938
:100C6000BF4FFE01E959FF4F808191818D939C9385
:100C7000FE01EF59FF4F808191810197F1F7FE014D
:100C8000EF59FF4F91838083E7E2F0E081E68083B4
:100C9000FE01E95AFF4F80E090E0A0EAB0E48083D3
:100CA0009183A283B3838E01035A1F4FFE01E95A39
:100CB000FF4F26E636E646E655E460817181828183
:100CC00093810E945C13DC01CB01F8018083918346
:100CD000A283B383FE01E35AFF4F20E030E040E8F7
:100CE0005FE360817181828193810E94E614882391
:100CF0000CF008C0FE01E55AFF4F81E090E09183BF
:100D0000808327C0FE01E35AFF4F20E03FEF4FE70B
:100D100057E460817181828193810E947A14181650
:100D20000CF006C0FE01E55AFF4F1182108211C07F
:100D30008E01055A1F4FFE01E35AFF4F60817181FA
:100D4000828193810E94AB11DC01CB01F801918378
:100D50008083DE01AB5ABF4FFE01E55AFF4F808111
:100D600091818D939C93FE01EB5AFF4F808191817D
:100D70000197F1F7FE01EB5AFF4F91838083E5E283
:100D8000F0E08081FE01E552FF4F99279183808337
:100D9000DE01AF51BF4FFE01E552FF4F80819181CF
:100DA0008C599F4F8D939C93FE01EF51FF4F808193
:100DB00091819F938F938CE691E09F938F93CE01C7
:100DC00084509F4F9F938F930E9496178DB79EB725
:100DD00006960FB6F8949EBF0FBE8DBFFE01E55B71
:100DE000FF4F80E090E0A0EAB0E480839183A2838B
:100DF000B3838E010F5A1F4FFE01E55BFF4F26E6BE
:100E000036E646E655E460817181828193810E94D5
:100E10005C13DC01CB01F80180839183A283B3834F
:100E2000FE01EF5AFF4F20E030E040E85FE36081D1
:100E30007181828193810E94E61488230CF008C09E
:100E4000FE01E15BFF4F81E090E09183808327C04A
:100E5000FE01EF5AFF4F20E03FEF4FE757E460817C
:100E60007181828193810E947A1418160CF006C059
:100E7000FE01E15BFF4F1182108211C08E01015B08
:100E80001F4FFE01EF5AFF4F608171818281938174
:100E90000E94AB11DC01CB01F80191838083DE015C
:100EA000A75BBF4FFE01E15BFF4F808191818D9376
:100EB0009C93FE01E75BFF4F808191810197F1F7E1
:100EC000FE01E75BFF4F9183808365E070E083E084
:100ED00090E00E94A50FFE01FF9680E090E0A0EA5E
:100EE000B0E480839183A283B3838E010B5B1F4F99
:100EF000FE01FF9626E636E646E655E460817181FE
:100F0000828193810E945C13DC01CB01F801808314
:100F10009183A283B383FE01EB5BFF4F20E030E0BF
:100F200040E85FE360817181828193810E94E614D1
:100F300088230CF008C0FE01ED5BFF4F81E090E0DC
:100F40009183808327C0FE01EB5BFF4F20E03FEFE2
:100F50004FE757E460817181828193810E947A1406
:100F600018160CF006C0FE01ED5BFF4F11821082D7
:100F700011C08E010D5B1F4FFE01EB5BFF4F6081C7
:100F80007181828193810E94AB11DC01CB01F80158
:100F900091838083FE01ED5BFF4F808191819EAF45
:100FA0008DAF8DAD9EAD0197F1F79EAF8DAFCE01A8
:100FB00084509F4F0E94800F80E090E0A0EAB0E450
:100FC0008BAB9CABADABBEAB26E636E646E655E456
:100FD0006BA97CA98DA99EA90E945C13DC01CB01A1
:100FE00089AF9AAFABAFBCAF20E030E040E85FE341
:100FF00069AD7AAD8BAD9CAD0E94E61488230CF0F0
:1010000005C081E090E098AF8FAB1AC020E03FEFC1
:101010004FE757E469AD7AAD8BAD9CAD0E947A1471
:1010200018160CF003C018AE1FAA0AC069AD7AAD3D
:101030008BAD9CAD0E94AB11DC01CB0198AF8FABA7
:101040008FA998AD9AAB89AB89A99AA90197F1F7B5
:101050009AAB89ABE7E2F0E080E6808380E090E045
:10106000A0EAB0E48FA398A7A9A7BAA726E636E618
:1010700046E655E46FA178A589A59AA50E945C1360
:10108000DC01CB018DA79EA7AFA7B8AB20E030E075
:1010900040E85FE36DA57EA58FA598A90E94E614A0
:1010A00088230CF005C081E090E09CA78BA71AC0B4
:1010B00020E03FEF4FE757E46DA57EA58FA598A9E7
:1010C0000E947A1418160CF003C01CA61BA60AC0B6
:1010D0006DA57EA58FA598A90E94AB11DC01CB015F
:1010E0009CA78BA78BA59CA59EA38DA38DA19EA13C
:1010F0000197F1F79EA38DA3E5E2F0E08081FE0168
:10110000E552FF4F992791838083DE01AF51BF4F96
:10111000FE01E552FF4F808191818C599F4F8D9345
:101120009C93FE01EF51FF4F808191819F938F939C
:101130008CE691E09F938F93CE0180509F4F9F93B9
:101140008F930E9496178DB79EB706960FB6F894A8
:101150009EBF0FBE8DBF80E090E0A0EAB0E48B8F11
:101160009C8FAD8FBE8F26E636E646E655E46B8D46
:101170007C8D8D8D9E8D0E945C13DC01CB0189A33B
:101180009AA3ABA3BCA320E030E040E85FE369A1F1
:101190007AA18BA19CA10E94E61488230CF005C0C3
:1011A00081E090E098A38F8F1AC020E03FEF4FE7D7
:1011B00057E469A17AA18BA19CA10E947A14181608
:1011C0000CF003C018A21F8E0AC069A17AA18BA1DE
:1011D0009CA10E94AB11DC01CB0198A38F8F8F8D56
:1011E00098A19A8F898F898D9A8D0197F1F79A8F9F
:1011F000898F6FE070E083E090E00E94A50F80E0AF
:1012000090E0A0EAB0E48F87988BA98BBA8B26E692
:1012100036E646E655E46F85788989899A890E9481
:101220005C13DC01CB018D8B9E8BAF8BB88F20E0E4
:1012300030E040E85FE36D897E898F89988D0E9458
:10124000E61488230CF005C081E090E09C8B8B8B2A
:101250001AC020E03FEF4FE757E46D897E898F8900
:10126000988D0E947A1418160CF003C01C8A1B8AF1
:101270000AC06D897E898F89988D0E94AB11DC012F
:10128000CB019C8B8B8B8B899C899E878D878D85D1
:101290009E850197F1F79E878D87CE0180509F4FE5
:1012A0000E94800F80E090E0A0EAB0E48B839C83F2
:1012B000AD83BE8326E636E646E655E46B817C8147
:1012C0008D819E810E945C13DC01CB0189879A8706
:1012D000AB87BC8720E030E040E85FE369857A8532
:1012E0008B859C850E94E61488230CF005C081E064
:1012F00090E098878F831AC020E03FEF4FE757E4D4
:1013000069857A858B859C850E947A1418160CF065
:1013100003C018861F820AC069857A858B859C85E3
:101320000E94AB11DC01CB0198878F838F81988558
:101330009A83898389819A810197F1F79A838983B6
:101340000C946A01CF93DF93CDB7DEB7E7E2F0E00C
:1013500080E68083E6E2F0E087EE8083DF91CF9144
:1013600008950F931F93CF93DF93CDB7DEB7CC567D
:10137000D0400FB6F894DEBF0FBECDBFFE01ED59D1
:10138000FF4F80E090E0A0E8BFE380839183A283D9
:10139000B3838E0107591F4FFE01ED59FF4F26E61B
:1013A00036E646E655E460817181828193810E9430
:1013B0005C13DC01CB01F80180839183A283B383AA
:1013C000FE01E759FF4F20E030E040E85FE3608135
:1013D0007181828193810E94E61488230CF008C0F9
:1013E000FE01E959FF4F81E090E09183808327C09F
:1013F000FE01E759FF4F20E03FEF4FE757E46081E0
:101400007181828193810E947A1418160CF006C0B3
:10141000FE01E959FF4F1182108211C08E01095956
:101420001F4FFE01E759FF4F6081718182819381D7
:101430000E94AB11DC01CB01F80191838083DE01B6
:10144000AF59BF4FFE01E959FF4F808191818D93C4
:101450009C93FE01EF59FF4F808191810197F1F735
:10146000FE01EF59FF4F9183808380E091E00E945D
:10147000800FFE01E95AFF4F80E090E0A0E8BFE353
:1014800080839183A283B3838E01035A1F4FFE0191
:10149000E95AFF4F26E636E646E655E4608171815B
:1014A000828193810E945C13DC01CB01F80180836F
:1014B0009183A283B383FE01E35AFF4F20E030E023
:1014C00040E85FE360817181828193810E94E6142C
:1014D00088230CF008C0FE01E55AFF4F81E090E040
:1014E0009183808327C0FE01E35AFF4F20E03FEF46
:1014F0004FE757E460817181828193810E947A1461
:1015000018160CF006C0FE01E55AFF4F118210823A
:1015100011C08E01055A1F4FFE01E35AFF4F608133
:101520007181828193810E94AB11DC01CB01F801B2
:1015300091838083DE01AB5ABF4FFE01E55AFF4F16
:10154000808191818D939C93FE01EB5AFF4F8081A6
:1015500091810197F1F7FE01EB5AFF4F9183808350
:1015600060E070E082E090E00E94A50FFE01E55B84
:10157000FF4F80E090E0A0E8BFE380839183A283E7
:10158000B3838E010F5A1F4FFE01E55BFF4F26E626
:1015900036E646E655E460817181828193810E943E
:1015A0005C13DC01CB01F80180839183A283B383B8
:1015B000FE01EF5AFF4F20E030E040E85FE360813A
:1015C0007181828193810E94E61488230CF008C007
:1015D000FE01E15BFF4F81E090E09183808327C0B3
:1015E000FE01EF5AFF4F20E03FEF4FE757E46081E5
:1015F0007181828193810E947A1418160CF006C0C2
:10160000FE01E15BFF4F1182108211C08E01015B70
:101610001F4FFE01EF5AFF4F6081718182819381DC
:101620000E94AB11DC01CB01F80191838083DE01C4
:10163000A75BBF4FFE01E15BFF4F808191818D93DE
:101640009C93FE01E75BFF4F808191810197F1F749
:10165000FE01E75BFF4F9183808384E591E00E9468
:10166000800FFE01FF9680E090E0A0E8BFE380835A
:101670009183A283B3838E010B5B1F4FFE01FF9604
:1016800026E636E646E655E46081718182819381E3
:101690000E945C13DC01CB01F80180839183A2835B
:1016A000B383FE01EB5BFF4F20E030E040E85FE3F7
:1016B00060817181828193810E94E61488230CF0FD
:1016C00008C0FE01ED5BFF4F81E090E091838083D5
:1016D00027C0FE01EB5BFF4F20E03FEF4FE757E4F1
:1016E00060817181828193810E947A1418160CF0B6
:1016F00006C0FE01ED5BFF4F1182108211C08E010A
:101700000D5B1F4FFE01EB5BFF4F6081718182819A
:1017100093810E94AB11DC01CB01F801918380839E
:10172000FE01ED5BFF4F808191819EAF8DAF8DAD4E
:101730009EAD0197F1F79EAF8DAF6AE070E082E059
:1017400090E00E94A50F80E090E0A0E8BFE38BABA3
:101750009CABADABBEAB26E636E646E655E46BA9E0
:101760007CA98DA99EA90E945C13DC01CB0189AFE5
:101770009AAFABAFBCAF20E030E040E85FE369ADCB
:101780007AAD8BAD9CAD0E94E61488230CF005C0A9
:1017900081E090E098AF8FAB1AC020E03FEF4FE7B9
:1017A00057E469AD7AAD8BAD9CAD0E947A141816E2
:1017B0000CF003C018AE1FAA0AC069AD7AAD8BAD9C
:1017C0009CAD0E94AB11DC01CB0198AF8FAB8FA910
:1017D00098AD9AAB89AB89A99AA90197F1F79AAB11
:1017E00089AB8AE591E00E94800F80E090E0A0E85C
:1017F000BFE38FA398A7A9A7BAA726E636E646E6D1
:1018000055E46FA178A589A59AA50E945C13DC0117
:10181000CB018DA79EA7AFA7B8AB20E030E040E892
:101820005FE36DA57EA58FA598A90E94E614882385
:101830000CF005C081E090E09CA78BA71AC020E0C7
:101840003FEF4FE757E46DA57EA58FA598A90E94AD
:101850007A1418160CF003C01CA61BA60AC06DA5AE
:101860007EA58FA598A90E94AB11DC01CB019CA796
:101870008BA78BA59CA59EA38DA38DA19EA101974F
:10188000F1F79EA38DA360E070E083E090E00E94FA
:10189000A50F80E090E0A0E8BFE38B8F9C8FAD8F19
:1018A000BE8F26E636E646E655E46B8D7C8D8D8D43
:1018B0009E8D0E945C13DC01CB0189A39AA3ABA38C
:1018C000BCA320E030E040E85FE369A17AA18BA1EE
:1018D0009CA10E94E61488230CF005C081E090E0F2
:1018E00098A38F8F1AC020E03FEF4FE757E469A11C
:1018F0007AA18BA19CA10E947A1418160CF003C047
:1019000018A21F8E0AC069A17AA18BA19CA10E9476
:10191000AB11DC01CB0198A38F8F8F8D98A19A8F8B
:10192000898F898D9A8D0197F1F79A8F898F80E63B
:1019300091E00E94800F80E090E0A0E8BFE38F87F5
:10194000988BA98BBA8B26E636E646E655E46F857A
:10195000788989899A890E945C13DC01CB018D8B7F
:101960009E8BAF8BB88F20E030E040E85FE36D895D
:101970007E898F89988D0E94E61488230CF005C01B
:1019800081E090E09C8B8B8B1AC020E03FEF4FE70B
:1019900057E46D897E898F89988D0E947A14181674
:1019A0000CF003C01C8A1B8A0AC06D897E898F894E
:1019B000988D0E94AB11DC01CB019C8B8B8B8B89AA
:1019C0009C899E878D878D859E850197F1F79E87DF
:1019D0008D876AE070E083E090E00E94A50F80E0D0
:1019E00090E0A0E8BFE38B839C83AD83BE8326E6B3
:1019F00036E646E655E46B817C818D819E810E94AE
:101A00005C13DC01CB0189879A87AB87BC8720E018
:101A100030E040E85FE369857A858B859C850E948C
:101A2000E61488230CF005C081E090E098878F834E
:101A30001AC020E03FEF4FE757E469857A858B8530
:101A40009C850E947A1418160CF003C018861F8219
:101A50000AC069857A858B859C850E94AB11DC0163
:101A6000CB0198878F838F8198859A838983898119
:101A70009A810197F1F79A83898386E691E00E9423
:101A8000800FC459DF4F0FB6F894DEBF0FBECDBF35
:101A9000DF91CF911F910F910895CF93DF93CDB731
:101AA000DEB7AE970FB6F894DEBF0FBECDBF9EA7D0
:101AB0008DA7EBE3F0E08DA59EA59595879595956F
:101AC000879595958795959587958064808380E027
:101AD00090E0A8E4B2E48CA39DA3AEA3BFA322E54B
:101AE00039E44DE950E46CA17DA18EA19FA10E9433
:101AF0005C13DC01CB0189A79AA7ABA7BCA720E0A8
:101B000030E040E85FE369A57AA58BA59CA50E941B
:101B1000E61488230CF003C081E088A718C020E0F9
:101B200030E04FE753E469A57AA58BA59CA50E94F8
:101B30007A1418160CF002C018A609C069A57AA577
:101B40008BA59CA50E94AB11DC01CB0188A788A5C1
:101B50008BA38BA18A95F1F78BA3EBE3F0E08DA526
:101B60009EA5959587959595879595958795959536
:101B70008795808380E090E0A0E8BFE3898F9A8F0B
:101B8000AB8FBC8F26E636E646E655E4698D7A8D46
:101B90008B8D9C8D0E945C13DC01CB018F8F98A3F1
:101BA000A9A3BAA320E030E040E85FE36F8D78A1FD
:101BB00089A19AA10E94E61488230CF005C081E057
:101BC00090E09E8F8D8F1AC020E03FEF4FE757E4E3
:101BD0006F8D78A189A19AA10E947A1418160CF031
:101BE00003C01E8E1D8E0AC06F8D78A189A19AA197
:101BF0000E94AB11DC01CB019E8F8D8F8D8D9E8D50
:101C0000988F8F8B8F89988D0197F1F7988F8F8B95
:101C1000EBE3F0E08DA58F708064808380E090E03E
:101C2000A8E4B2E48E879F87A88BB98B22E539E4BC
:101C30004DE950E46E857F85888999890E945C13FF
:101C4000DC01CB018B8B9C8BAD8BBE8B20E030E01D
:101C500040E85FE36B897C898D899E890E94E61448
:101C600088230CF003C081E08A8B18C020E030E0AC
:101C70004FE753E46B897C898D899E890E947A1491
:101C800018160CF002C01A8A09C06B897C898D89EC
:101C90009E890E94AB11DC01CB018A8B8A898D87DA
:101CA0008D858A95F1F78D87EBE3F0E08DA58F7038
:101CB000808380E090E0A0EAB0E48B839C83AD83D6
:101CC000BE8326E636E646E655E46B817C818D814F
:101CD0009E810E945C13DC01CB0189879A87AB87C8
:101CE000BC8720E030E040E85FE369857A858B853A
:101CF0009C850E94E61488230CF005C081E090E0EA
:101D000098878F831AC020E03FEF4FE757E469853B
:101D10007A858B859C850E947A1418160CF003C076
:101D200018861F820AC069857A858B859C850E94EA
:101D3000AB11DC01CB0198878F838F8198859A83C3
:101D4000898389819A810197F1F79A838983AE9675
:101D50000FB6F894DEBF0FBECDBFDF91CF910895CF
:101D6000CF93DF93CDB7DEB781E090E00E944D0DB9
:101D700010928D0110928C01DF91CF910895CF9335
:101D8000DF93CDB7DEB768970FB6F894DEBF0FBE0E
:101D9000CDBF80E090E0A0E7B1E48F87988BA98B5E
:101DA000BA8B26E636E646E655E46F85788989895A
:101DB0009A890E945C13DC01CB018D8B9E8BAF8BCB
:101DC000B88F20E030E040E85FE36D897E898F893D
:101DD000988D0E94E61488230CF005C081E090E005
:101DE0009C8B8B8B1AC020E03FEF4FE757E46D8947
:101DF0007E898F89988D0E947A1418160CF003C082
:101E00001C8A1B8A0AC06D897E898F89988D0E94E1
:101E1000AB11DC01CB019C8B8B8B8B899C899E87C2
:101E20008D878D859E850197F1F79E878D8783E34A
:101E300090E00E944D0D80E090E0A0E8BFE38B832E
:101E40009C83AD83BE8326E636E646E655E46B8189
:101E50007C818D819E810E945C13DC01CB0189878E
:101E60009A87AB87BC8720E030E040E85FE3698574
:101E70007A858B859C850E94E61488230CF005C02A
:101E800081E090E098878F831AC020E03FEF4FE712
:101E900057E469857A858B859C850E947A1418168B
:101EA0000CF003C018861F820AC069857A858B856D
:101EB0009C850E94AB11DC01CB0198878F838F81B9
:101EC00098859A83898389819A810197F1F79A830A
:101ED000898382E390E00E944D0D88E290E00E94A9
:101EE0004D0D8CE090E00E944D0D0E94B00E689662
:101EF0000FB6F894DEBF0FBECDBFDF91CF9108952E
:101F0000CF93DF93CDB7DEB722970FB6F894DEBF3D
:101F10000FBECDBF9A8389830AC0E981FA8180818F
:101F20000E942C1089819A8101969A838983E98184
:101F3000FA818081882389F722960FB6F894DEBF54
:101F40000FBECDBFDF91CF910895CF93DF93CDB773
:101F5000DEB724970FB6F894DEBF0FBECDBF9A83CD
:101F600089837C836B8389819A819C01220F331F33
:101F7000220F331FC901880F991F880F991F280F3F
:101F8000391F8B819C81820F931F90938D018093C9
:101F90008C0180918C0190918D01843191053CF4EC
:101FA00080918C0190918D0180680E944D0D8091EF
:101FB0008C0190918D0184319105ACF080918C0160
:101FC00090918D018832910574F480918C019091EB
:101FD0008D0124E130E0B9010E94DC1A805C9F4F42
:101FE00080680E944D0D80918C0190918D01883206
:101FF0009105A4F080918C0190918D018C33910515
:102000006CF480918C0190918D0128E230E0B9014F
:102010000E94DC1A449680680E944D0D80918C01CC
:1020200090918D018D33910574F080918C01909188
:102030008D012CE330E0B9010E94DC1A8C5A9F4FCD
:1020400080680E944D0D24960FB6F894DEBF0FBE37
:10205000CDBFDF91CF910895CF93DF93CDB7DEB79A
:10206000A9970FB6F894DEBF0FBECDBF89A78091A8
:102070008C0190918D018431910521F480EC90E0E8
:102080000E944D0D80918C0190918D0188329105B7
:1020900021F484E990E00E944D0D80918C01909193
:1020A0008D018C33910521F484ED90E00E944D0D5B
:1020B000EBE3F0E089A58595859585958595806507
:1020C000808380E090E0A8E4B2E488A399A3AAA367
:1020D000BBA322E539E44DE950E468A179A18AA1C6
:1020E0009BA10E945C13DC01CB018DA39EA3AFA337
:1020F000B8A720E030E040E85FE36DA17EA18FA1AA
:1021000098A50E94E61488230CF003C081E08CA3FC
:1021100018C020E030E04FE753E46DA17EA18FA10D
:1021200098A50E947A1418160CF002C01CA209C0CF
:102130006DA17EA18FA198A50E94AB11DC01CB01FE
:102140008CA38CA18F8F8F8D8A95F1F78F8FEBE306
:10215000F0E089A585958595859585958061808335
:1021600080E090E0A8E4B2E48E8B9F8BA88FB98FBB
:1021700022E539E44DE950E46E897F89888D998D97
:102180000E945C13DC01CB018B8F9C8FAD8FBE8FC7
:1021900020E030E040E85FE36B8D7C8D8D8D9E8D7F
:1021A0000E94E61488230CF003C081E08A8F18C0D7
:1021B00020E030E04FE753E46B8D7C8D8D8D9E8D5C
:1021C0000E947A1418160CF002C01A8E09C06B8D8A
:1021D0007C8D8D8D9E8D0E94AB11DC01CB018A8F91
:1021E0008A8D8D8B8D898A95F1F78D8BEBE3F0E0ED
:1021F00089A58F708065808380E090E0A8E4B2E4D8
:102200008C879D87AE87BF8722E539E44DE950E48E
:102210006C857D858E859F850E945C13DC01CB01DA
:10222000898B9A8BAB8BBC8B20E030E040E85FE37E
:1022300069897A898B899C890E94E61488230CF02D
:1022400003C081E0888B18C020E030E04FE753E402
:1022500069897A898B899C890E947A1418160CF0F6
:1022600002C0188A09C069897A898B899C890E9471
:10227000AB11DC01CB01888B88898B878B858A9594
:10228000F1F78B87EBE3F0E089A58F7080618083A5
:1022900080E090E0A8E4B2E48A839B83AC83BD83B2
:1022A00022E539E44DE950E46A817B818C819D818E
:1022B0000E945C13DC01CB018F839887A987BA87C2
:1022C00020E030E040E85FE36F81788589859A857A
:1022D0000E94E61488230CF003C081E08E8318C0AE
:1022E00020E030E04FE753E46F81788589859A8557
:1022F0000E947A1418160CF002C01E8209C06F8169
:10230000788589859A850E94AB11DC01CB018E838B
:102310008E81898389818A95F1F7898380918C01E7
:1023200090918D01019690938D0180938C01809105
:102330008C0190918D018035910521F410928D01D1
:1023400010928C01A9960FB6F894DEBF0FBECDBFD8
:10235000DF91CF910895EF92FF920F931F937B012E
:102360008C0120E030E040E05FE40E94B01488235C
:102370007CF020E030E040E05FE4C801B7010E945B
:10238000FE120E941C15605070408040904804C0AE
:10239000C801B7010E941C151F910F91FF90EF908B
:1023A0000895A0E0B0E0E7EDF1E10C94071BFC011B
:1023B0006A019081923008F41BC1DB018C9182305C
:1023C00080F0943061F4843009F012C19181EB0106
:1023D0008981981709F40CC1E4E8F1E009C184305F
:1023E00011F4FB0105C1823091F4923009F000C173
:1023F000EA01DF0188E00D9009928150E1F78181C7
:10240000FB0191818923E6018983F601F1C09230B5
:1024100041F362807380EB018A809B80E480F580C9
:10242000068117812C813D814E815F815301A8185F
:10243000B908C501B7FCABC080970CF457C086142F
:1024400097040CF4BEC03401EE24FF24870191816F
:10245000FB018181981709F4A6C0992309F49CC057
:102460002E193F09400B510B57FDB0C0E6011982F0
:102470007B826A82F6012483358346835783E60193
:102480002C813D814E815F8179018A01DA01C90188
:102490000197A109B1098F5F9F4FAF4FBF43F8F478
:1024A000E6016A817B81A8019701220F331F441F37
:1024B000551F6150704079018A01DA01C901019705
:1024C000A109B1098F5F9F4FAF4FBF4360F3E60192
:1024D0007B836A83F601248335834683578383E0B5
:1024E000D6018C9357FD39C0F60182C0861497043B
:1024F000B4F4C0E0D0E0DA01C90181709070A0703E
:10250000B0705695479537952795282B392B4A2B30
:102510005B2B2196AC16BD0671F78A0C9B1C6814C8
:1025200079040CF094CFC0E0D0E05401A618B708AD
:10253000D801C70181709070A070B0701695079592
:10254000F794E794E82AF92A0A2B1B2B2196AC165C
:10255000BD0671F76A0C7B1C7ACFDA01C901B6950A
:10256000A795979587952170307040705070282BF3
:10257000392B4A2B5B2BE6012C833D834E835F83F3
:102580008A819B8101969B838A83F60131C08827CB
:1025900099278A199B0950CFE21AF30A040B150BED
:1025A000A801970161CFE60199837B826A822E0D93
:1025B0003F1D401F511FF6012483358346835783F7
:1025C0008ECF20E030E040E050E041CF81E0E601F6
:1025D00089837B826A8250954095309521953F4F43
:1025E0004F4F5F4FF601248335834683578347CF90
:1025F000CF01EEE0CDB7DEB70C94231BA0E2B0E034
:10260000E4E0F3E10C940F1B69837A838B839C8352
:102610002D833E834F83588789E1E82EF12CEC0E01
:10262000FD1EB701CE0101960E948E168E010F5E2F
:102630001F4FB801CE0105960E948E168A8991E03F
:1026400089278A8BAE01475F5F4FB801C7010E949F
:10265000D1110E946C15E6E0A0960C942B1BA0E211
:10266000B0E0E5E3F3E10C940F1B69837A838B837D
:102670009C832D833E834F83588799E1E92EF12C6B
:10268000EC0EFD1EB701CE0101960E948E168E0142
:102690000F5E1F4FB801CE0105960E948E16AE0147
:1026A000475F5F4FB801C7010E94D1110E946C15AE
:1026B000E6E0A0960C942B1BA0E2B0E0E2E6F3E18A
:1026C0000C94031B69837A838B839C832D833E83C5
:1026D0004F8358878E01075E1F4FB801CE010196C8
:1026E0000E948E16F1E1EF2EF12CEC0EFD1EB701CB
:1026F000CE0105960E948E16898D823078F09989D8
:10270000923040F420E09A8D8A89981321E02A8B38
:10271000B701E9C0843051F4923061F020E09A8D25
:102720008A89981321E02A8FB801DDC0943029F4FA
:10273000823041F764E871E0D6C0823079F392309C
:1027400009F32D8D3E8D4F8D58A18D899E89AF89BE
:10275000B88D222433242101AA24BB246501EE2450
:10276000FF24870160E070E00DC06F5F7F4F603233
:10277000710599F1880F991FAA1FBB1F56954795A0
:102780003795279520FF19C0280E391E4A1E5B1E5B
:10279000662477244301281639064A065B0628F486
:1027A000E1E06E2E712C812C912CAE0CBF1CC01E52
:1027B000D11EA60CB71CC81CD91CEE0CFF1C001F98
:1027C000111FB7FFD2CFE1E06E2E712C812C912C1E
:1027D000E628F72808291929C8CF8B8D9C8D2B89CD
:1027E0003C89820F931F02969C878B871A869A8D4D
:1027F0008A89981711F081E08A87D7FE17C08B85E8
:102800009C85A0FE0CC0569447943794279420E0F2
:1028100030E040E050E8222A332A442A552AD69450
:10282000C794B794A79401969C878B8730E0A31632
:1028300030E0B30630E0C30630E4D30618F58B85EC
:102840009C850EC0220C331C441C551C019720E0B3
:10285000A21620E0B20620E0C20620E4D20680F4F0
:10286000AA0CBB1CCC1CDD1C57FEECCF31E0632E48
:10287000712C812C912CA628B728C828D928E2CF02
:102880009C878B87D601C5018F779070A070B07040
:1028900080349105A105B10551F0AD86BE86CF8685
:1028A000D88A83E08987BE01675F7F4F1CC0A7FC81
:1028B000F4CF211431044104510479F380E490E011
:1028C000A0E0B0E0A80EB91ECA1EDB1E80E8682E8C
:1028D0008FEF782E8FEF882E8FEF982EA620B720BF
:1028E000C820D920DACFCB010E946C15E2E1A09676
:1028F0000C941F1BA8E1B0E0E0E8F4E10C940F1B7E
:1029000069837A838B839C832D833E834F8358878F
:1029100081E1E82EF12CEC0EFD1EB701CE010196EF
:102920000E948E168E01075F1F4FB801CE010596DB
:102930000E948E168989823018F42FEF3FEF0BC06A
:1029400089858230D0F3B801C7010E942D17282F46
:10295000332727FD3095C901E6E068960C942B1BC0
:10296000A8E1B0E0E6EBF4E10C940F1B69837A83F5
:102970008B839C832D833E834F83588781E1E82E90
:10298000F12CEC0EFD1EB701CE0101960E948E16B1
:102990008E01075F1F4FB801CE0105960E948E166B
:1029A0008989823018F42FEF3FEF0BC08985823080
:1029B000D0F3B801C7010E942D17282F332727FD18
:1029C0003095C901E6E068960C942B1BA8E1B0E0B5
:1029D000ECEEF4E10C940F1B69837A838B839C8368
:1029E0002D833E834F83588781E1E82EF12CEC0E36
:1029F000FD1EB701CE0101960E948E168E01075F63
:102A00001F4FB801CE0105960E948E16898982302B
:102A100018F08985823018F421E030E008C0B80150
:102A2000C7010E942D17282F332727FD3095C90194
:102A3000E6E068960C942B1BACE0B0E0E2E2F5E136
:102A40000C94131B69837A838B839C83BE016B5F19
:102A50007F4FCE0101960E948E168D81823061F0EB
:102A6000823050F0843069F48E81882359F52FEF3D
:102A70003FEF4FEF5FE72AC020E030E040E050E05A
:102A800025C02F81388537FDF7CF2F31310564F709
:102A90008EE190E0821B930B29853A854B855C85FE
:102AA00004C056954795379527958A95D2F78E811C
:102AB000882361F050954095309521953F4F4F4FB9
:102AC0005F4F04C020E030E040E050E8CA01B901A7
:102AD000E2E02C960C942F1B4F925F926F927F92A4
:102AE0008F929F92AF92BF92DF92EF92FF920F93DD
:102AF0001F9320E030E040E050E0FC01E480F580EE
:102B000006811781D1808081823038F4D801C701D5
:102B1000A061AF77B0706FEFD9C0843009F46EC098
:102B2000823009F471C0E114F1040105110509F4C2
:102B30006BC0828193816FEF823896070CF06AC078
:102B400062E87FEF681B790B6A3171050CF080C079
:102B500047015801062E04C0B694A7949794879411
:102B60000A94D2F744245524320181E090E0A0E099
:102B7000B0E004C0880F991FAA1FBB1F6A95D2F747
:102B80000197A109B109E822F9220A231B23E114C4
:102B9000F1040105110529F061E0462E512C612C4C
:102BA000712C85017401E428F52806291729D8011C
:102BB000C7018F779070A070B07080349105A10527
:102BC000B10509F457C0D801C701CF96A11DB11DA9
:102BD00060E070E08030E0E09E07E0E0AE07E0E417
:102BE000BE0710F061E070E027E0B695A7959795D5
:102BF00087952A95D1F7AF77B07068C080E090E0F4
:102C0000A0E0B0E06FEF62C080E090E0A0E0B0E054
:102C100060E05CC0803891058CF7BC0161587F4F43
:102C2000D801C7018F779070A070B0708034910583
:102C3000A105B105A1F08FE390E0A0E0B0E0E80EBF
:102C4000F91E0A1F1B1F17FD28C0D801C701CCCFD2
:102C500060E070E080E090E0A0E0B0E0CCCFE7FE84
:102C6000F2CF80E490E0A0E0B0E0E80EF91E0A1F89
:102C70001B1FE9CFE7FC18C080E090E060E0E6169B
:102C800060E0F60660E0060760E4160710F081E0F9
:102C900090E0BC01D801C701A7CF16950795F7941E
:102CA000E7946F5F7F4FD1CFD801C701805C9F4F02
:102CB000AF4FBF4F60E070E08030E0E09E07E0E0A3
:102CC000AE07E0E4BE0708F48FCF8CCF282F392F52
:102CD0009A2F9F77842F8078892B962F9795992705
:102CE00097958F77482F492B6695852F8078862B6F
:102CF000D794DD24D7948F77582F5D29CA01B90165
:102D00001F910F91FF90EF90DF90BF90AF909F9039
:102D10008F907F906F905F904F900895FC01DB0142
:102D2000208131819281492F4F7750E0991F992757
:102D3000991F8381682F660F692B881F8827881F3A
:102D4000FD018183662309F049C021153105410544
:102D5000510509F470C082E89FEFFD0193838283DF
:102D6000220F331F441F551F220F331F441F551FAF
:102D7000220F331F441F551F220F331F441F551F9F
:102D8000220F331F441F551F220F331F441F551F8F
:102D9000220F331F441F551F83E08C932030F0E037
:102DA0003F07F0E04F07F0E45F0790F482E89FEF01
:102DB000220F331F441F551F0197203060E0360754
:102DC00060E0460760E4560798F3FD019383828331
:102DD000FD01248335834683578308956F3F71F146
:102DE000862F99278F579040FD019383828383E03C
:102DF0008C93220F331F441F551F220F331F441F74
:102E0000551F220F331F441F551F220F331F441F0E
:102E1000551F220F331F441F551F220F331F441FFE
:102E2000551F220F331F441F551F506424833583C1
:102E300046835783089582E08C93089521153105C8
:102E40004105510519F484E08C93089544FD02C0B6
:102E50001C92BECF81E08C93BBCFEF92FF920F9379
:102E60001F93CF93DF93FC01DB018081823050F010
:102E70009C91923038F0843041F49430B1F08181EB
:102E8000882381F461E070E04BC09430E9F1823036
:102E9000A1F09230A1F36181ED018981681791F071
:102EA000662381F36FEF7FEF3BC0EB018981682FD1
:102EB00077278181681B710933C0923059F560E032
:102EC00070E02EC022813381ED018A819B818217BF
:102ED000930734F3281739079CF0E480F5800681C6
:102EE0001781FD0124813581468157812E153F05CB
:102EF00040075107A8F2E216F30604071507F8F693
:102F0000662309F0BFCFCECFFB018181882309F072
:102F1000B9CFC8CFEB018981882309F0B3CFC2CFE5
:102F2000CB01E6E0CDB7DEB70C942B1B0F931F93BC
:102F3000CF93DF93CDB7DEB760970FB6F894DEBFBF
:102F40000FBECDBF0F89188D86E08E831C830B8347
:102F50008FEF9FE798878F83AE01455E5F4F5A835F
:102F60004983698D7A8DCE0103960E94C817298501
:102F70003A85020F131FF801108260960FB6F8947D
:102F8000DEBF0FBECDBFDF91CF911F910F9108958E
:102F90002F923F924F925F926F927F928F929F9269
:102FA000AF92BF92CF92DF92EF92FF920F931F9357
:102FB000CF93DF93CDB7DEB764970FB6F894DEBF3B
:102FC0000FBECDBFCC24DD2476011C017C8B6B8B26
:102FD0002A01FC0117821682838181FD03C08FEFD5
:102FE0009FEF85C2AA24BB246FC2A0FE54C28A8967
:102FF00080538A30E8F4FA89F03341F42D85222396
:1030000029F4A3FC03C080E091E06FC08AE0ED8565
:10301000E802C0011124FA89F80FF053FD87F7FF89
:1030200002C02FE72D87A3FC49C23D853E8746C2DB
:10303000C50188709070A3FE05C0ED85EE2311F4E4
:10304000F1E0FD872A89283624F525360CF05BC08F
:10305000233509F480C024358CF42B32C1F12C3295
:1030600034F42032C1F1233209F00AC23CC03A895B
:103070003D32B1F13E3209F003C23AC08A8983364B
:1030800009F449C084360CF081C0883509F0F8C1D4
:103090001BC0EA89E03709F4A3C0E13744F4EC36F9
:1030A00069F1EF3671F0E93609F0EAC16FC0FA89CB
:1030B000F53709F49DC0F83739F0F33709F0E0C16E
:1030C00034C028E0298B94C030E1398B91C080E175
:1030D00090E0A82AB92AE0E2F0E0AE2ABF2AEEC1C9
:1030E00020E830E00DC080E490E0A82AB92AE6C1CB
:1030F000E8E0F0E0AE2ABF2A1D86E0C124E030E01F
:10310000A22AB32ADBC13FE3C32E3E8531503E875E
:1031100083E68A8B41C1F201C080FE85F150FE87B3
:1031200022E030E0420E531E37C1F201C080D18050
:10313000892B49F0FD856F2F772767FD7095C601B4
:103140000E94A41A19C0F60101900020E9F73197F6
:10315000EC19E98B12C0F201C080D180892B49F0B3
:10316000FD856F2F772767FD7095C6010E94991A1C
:1031700003C0C6010E94901A898B22E030E0420E03
:10318000531E3E858989381B3E8706C1A2FE08C0B2
:10319000F20180819181A281B38124E030E009C0F5
:1031A000F20180819181AA2797FDA095BA2F22E094
:1031B00030E0420E531E6C017D01B7FF0CC082E06F
:1031C00090E0A82AB92AF094E094D094C094C11C4D
:1031D000D11CE11CF11CEFEBFFEFAE22BF2221C09E
:1031E00020E430E0A22AB32A38E73A8B80E1898BC9
:1031F000A2FE08C0F20180819181A281B38124E006
:1032000030E007C0F20180819181AA27BB2722E02C
:1032100030E0420E531E6C017D018FEC9FEFA8221F
:10322000B92287017601FE013196F88BEF87F98983
:103230006F2E772488249924C801B701A401930133
:103240000E943A1B6A3024F02A89620F615201C041
:10325000605DEF85F8896193F88BEF87C801B7014E
:10326000A40193010E943A1B79018A0121153105BD
:103270004105510509F7CC24DD247601CE010196E4
:10328000CF84C81AC50182739070892B19F0FE850E
:10329000F150FE87A6FE09C02989203111F482E091
:1032A00001C081E03E85381B3E8728E0822E912CAC
:1032B0008A209B20A3FE18C08D85282F332727FD49
:1032C00030958C2D9927821793073CF0E7EFFFEF9D
:1032D000AE22BF228824992407C0FD85FC19FD87F2
:1032E0002E852F1B2E8703C03E853C193E87C501C6
:1032F00080789170892B69F48E8506C0B10180E2D7
:1033000090E00E94AF1A812F182F11501816B4F3B5
:103310001E87A1FE04C0B1018DE290E00BC0A4FEA7
:1033200004C0B1018BE290E005C0A5FE05C0B1016B
:1033300080E290E00E94AF1AA6FE10C0B10180E3C7
:1033400090E00E94AF1A8989803141F4B101EA8985
:103350008E2F992787FD90950E94AF1AB0FE0DC061
:103360008E8506C0B10180E390E00E94AF1A812FE4
:10337000182F11501816B4F31E87892869F02D856F
:1033800006C0B10180E390E00E94AF1A212F122FF6
:1033900011501216B4F31D8790E8692E712C6A2023
:1033A0007B20A7FC0DC08E8506C0B10180E290E0B5
:1033B0000E94AF1A812F182F11501816B4F31E87D0
:1033C000FA89F33641F4B1018C2D992787FD909548
:1033D0000E94AF1A45C02A892337B1F4460156012D
:1033E000198909C0F50181915F01B101992787FD14
:1033F00090950E94AF1A1150A8F76401F989CF0E79
:10340000D11C2FEF298B2CC03A89333519F00F8549
:1034100018891FC046018601B98808C0F801849147
:10342000B10199270E94AF1A0F5F1F4FBA94FFEFA7
:10343000BF16A1F764012989C20ED11CF98B10C0F7
:10344000F80182918F01B101992787FD90950E9423
:10345000AF1ACE0101960817190791F7188B0F873D
:103460006728B1F08E8506C0B10180E290E00E942D
:10347000AF1A812F182F11501816B4F31E8708C0E9
:10348000B101FA898F2F992787FD90950E94AF1A75
:10349000AA24BB2413C02A89253241F43AE0398B8F
:1034A0001E861D8681E0A82EB12C08C0B101EA89D4
:1034B0008E2F992787FD90950E94AF1A2B893C8902
:1034C0002F5F3F4F3C8B2B8BF101838183FF04C027
:1034D000EB89FC89F49103C0EB89FC89F081FA8BBC
:1034E0002A89222309F081CDF10186819781649692
:1034F0000FB6F894DEBF0FBECDBFDF91CF911F9105
:103500000F91FF90EF90DF90CF90BF90AF909F9082
:103510008F907F906F905F904F903F902F90089585
:10352000FC0105900020E9F7809590958E0F9F1F74
:103530000895FC010590615070400110D8F7809506
:1035400090958E0F9F1F0895FC016150704001906F
:103550000110D8F7809590958E0F9F1F08950F93B7
:103560001F93CF93DF938C01EB018B81992781FF10
:103570001BC082FF0DC02E813F818C819D81281749
:10358000390764F4E881F9810193F983E88306C07F
:10359000E885F985802F0995892B31F48E819F81EB
:1035A00001969F838E8302C00FEF1FEFC801DF914A
:1035B000CF911F910F91089597FB092E07260AD0EE
:1035C00077FD04D00CD006D000201AF470956195D8
:1035D0007F4F0895F6F7909581959F4F0895AA1B08
:1035E000BB1B51E107C0AA1FBB1FA617B70710F0EE
:1035F000A61BB70B881F991F5A95A9F78095909520
:10360000BC01CD0108952F923F924F925F926F922D
:103610007F928F929F92AF92BF92CF92DF92EF9262
:10362000FF920F931F93CF93DF93CDB7DEB7CA1BE3
:10363000DB0B0FB6F894DEBF0FBECDBF09942A880E
:10364000398848885F846E847D848C849B84AA84B6
:10365000B984C884DF80EE80FD800C811B81AA8143
:10366000B981CE0FD11D0FB6F894DEBF0FBECDBF0E
:10367000ED010895A1E21A2EAA1BBB1BFD010DC08E
:10368000AA1FBB1FEE1FFF1FA217B307E407F50712
:1036900020F0A21BB30BE40BF50B661F771F881FEE
:1036A000991F1A9469F760957095809590959B0184
:0836B000AC01BD01CF0108953A
:1036B80054657374696E672053656E736F72730017
:1036C80000000000004952204F6E0000000000007A
:1036D80000000000000000000000536F6E617220BF
:1036E8004F6E0000000000000000000000000043D2
:1036F8006F646520436F6D706C6574650000000031
:10370800000000004C49523D20005249523D200023
:103718004C534F3D200052534F3D20002564005725
:10372800726F6E67206F757470757400000000000A
:0C37380000000000000000000000000085
:00000001FF
